:020000040000FA
:04080000E7EF07F027
:1008100003B213EF05F0F2B42EEF05F09EB036EF01
:1008200005F09EB23EEF05F0F2A81AEF04F0F2B226
:1008300025EF04F0F2A620EF04F0F2B022EF04F06E
:1008400096EF07F0F296F290FF00CD90F2929EA004
:100850002FEF04F00101533F2FEF04F0542BAEC1F2
:10086000B2F1AFC1B3F1B0C1B4F1B1C1B5F1AAC138
:10087000AEF1ABC1AFF1ACC1B0F1ADC1B1F1A6C148
:10088000AAF1A7C1ABF1A8C1ACF1A9C1ADF1A2C158
:10089000A6F1A3C1A7F1A4C1A8F1A5C1A9F19EC168
:1008A000A2F19FC1A3F1A0C1A4F1A1C1A5F19AC178
:1008B0009EF19BC19FF19CC1A0F19DC1A1F196C188
:1008C0009AF197C19BF198C19CF199C19DF1CECF4E
:1008D00096F1CFCF97F153C198F154C199F1CF6AF6
:1008E000CE6A0101536B546B9E90CD800FBC0F8E6E
:1008F0000FBA7EEF04F00F8A96EF07F00F8C0FBE51
:10090000BAEF04F096C19AF197C19BF198C19CF19E
:1009100099C19DF19AC19EF19BC19FF19CC1A0F12B
:100920009DC1A1F19EC1A2F19FC1A3F1A0C1A4F1FB
:10093000A1C1A5F1A2C1A6F1A3C1A7F1A4C1A8F1CB
:10094000A5C1A9F1A6C1AAF1A7C1ABF1A8C1ACF19B
:10095000A9C1ADF1AAC1AEF1ABC1AFF1ACC1B0F16B
:10096000ADC1B1F1AEC1B2F1AFC1B3F1B0C1B4F13B
:10097000B1C1B5F101015E6B5F6B606B616B96514C
:100980005E2797515F2398516023995161239A51B3
:100990005E279B515F239C5160239D5161239E5193
:1009A0005E279F515F23A0516023A1516123A25173
:1009B0005E27A3515F23A4516023A5516123A65153
:1009C0005E27A7515F23A8516023A9516123AA5133
:1009D0005E27AB515F23AC516023AD516123AE5113
:1009E0005E27AF515F23B0516023B1516123B251F3
:1009F0005E27B3515F23B4516023B5516123D89072
:100A00000101613360335F335E33D890010161339C
:100A100060335F335E33D8900101613360335F33FD
:100A20005E3396EF07F00392030103EE00F080516E
:100A30007F0BE92604C0EFFF802B8151805D700B96
:100A4000D8A48B8200008051815D700BD8A48B925A
:100A500081518019D8B4079096EF07F0F294010104
:100A6000453F96EF07F0462B96EF07F09E90010169
:100A7000533F96EF07F0542B96EF07F09E92040039
:100A800062A143EF05F0077C07AC5EEF05F0C2748E
:100A9000C2B458EF05F0C3CFB3F5C4CFB4F5050128
:100AA000D890B433B333D890B433B3335FEF05F099
:100AB000C3CF55F1C4CF56F15FEF05F0C28207B442
:100AC000CCEF05F047C14BF148C14CF149C14DF1A4
:100AD0004AC14EF15EC162F15FC163F160C164F170
:100AE00061C165F196C1B6F197C1B7F198C1B8F18E
:100AF00099C1B9F19AC1BAF19BC1BBF19CC1BCF1DA
:100B00009DC1BDF19EC1BEF19FC1BFF1A0C1C0F1A9
:100B1000A1C1C1F1A2C1C2F1A3C1C3F1A4C1C4F179
:100B2000A5C1C5F1A6C1C6F1A7C1C7F1A8C1C8F149
:100B3000A9C1C9F1AAC1CAF1ABC1CBF1ACC1CCF119
:100B4000ADC1CDF1AEC1CEF1AFC1CFF1B0C1D0F1E9
:100B5000B1C1D1F1B2C1D2F1B3C1D3F1B4C1D4F1B9
:100B6000B5C1D5F1B3C5B5F5B4C5B6F5B5C5B7F5DD
:100B7000B6C5B8F5010155515B2756515C23E86AAB
:100B80005D230E2ECCEF05F05CC157F15DC158F12D
:100B90005B6B5C6B5D6B078E0201002F96EF07F0BD
:100BA0003C0E006F00C10CF101C10DF102C10EF14C
:100BB00003C10FF104C110F105C111F106C112F119
:100BC00007C113F108C114F109C115F10AC116F1E9
:100BD0000BC117F134C135F105012F51000AD8B40A
:100BE00095EF06F005012F51010AD8B41FEF06F06A
:100BF00005012F51020AD8B460EF06F005012F510C
:100C0000030AD8B460EF06F005012F51040AD8B4E6
:100C100060EF06F005012F51050AD8B460EF06F029
:100C200005012F51060AD8B460EF06F005012F51D7
:100C3000070AD8B460EF06F02F6B95EF06F00501B8
:100C400053672AEF06F054672AEF06F055672AEF3C
:100C500006F056672EEF06F095EF06F057C500F147
:100C600058C501F159C502F15AC503F10101010E40
:100C7000046F000E056F000E066F000E076F1EEC6E
:100C800022F000C157F501C158F502C159F503C161
:100C90005AF5006753EF06F0016753EF06F002675D
:100CA00053EF06F0036795EF06F053C557F554C5AB
:100CB00058F555C559F556C55AF50F8895EF06F004
:100CC0000501306766EF06F095EF06F00FBE7BEF8B
:100CD00006F010A080EF06F00101476777EF06F0FD
:100CE000486777EF06F0496777EF06F04A677BEFD2
:100CF00006F080EF06F007AE80EF06F092EF06F008
:100D00000501312F95EF06F03C0E316F302F95EF36
:100D100006F00101000E626FE00E636FA50E646FB6
:100D2000010E656F0501306B0F880501626B33B7EB
:100D30009BEF06F062810CC100F10DC101F10EC103
:100D400002F10FC103F110C104F111C105F112C18B
:100D500006F113C107F114C108F115C109F116C15B
:100D60000AF117C10BF135C134F100C10CF101C119
:100D70000DF102C10EF103C10FF104C110F105C163
:100D800011F106C112F107C113F108C114F109C133
:100D900015F10AC116F10BC117F134C135F101018A
:100DA0008A67DAEF06F08B67DAEF06F08C67DAEF26
:100DB00006F08D67DEEF06F00EEF07F08EC100F152
:100DC0008FC101F190C102F191C103F10101010E46
:100DD000046F000E056F000E066F000E076F1EEC0D
:100DE00022F000C18EF101C18FF102C190F103C167
:100DF00091F1006703EF07F0016703EF07F0026767
:100E000003EF07F003670EEF07F08AC18EF18BC185
:100E10008FF18CC190F18DC191F10F80D57ED5BE3F
:100E200069D0D6CF47F1D7CF48F145C149F1E86A3B
:100E3000E8CF4AF1109047C100F148C101F149C122
:100E400002F14AC103F101010A0E046F000E056FA1
:100E5000000E066F000E076F1EEC22F000AF108030
:100E6000010154A740EF07F00F9A0F9C0F9E01015C
:100E7000000E5E6F600E5F6F3D0E606F080E616F5B
:100E8000010147BF50EF07F0486750EF07F049678F
:100E900050EF07F04A6750EF07F0F28875EF07F060
:100EA000F2985E6B5F6B606B616B966B976B986B88
:100EB000996B9A6B9B6B9C6B9D6B9E6B9F6BA06BF6
:100EC000A16BA26BA36BA46BA56BA66BA76BA86BA6
:100ED000A96BAA6BAB6BAC6BAD6BAE6BAF6BB06B56
:100EE000B16BB26BB36BB46BB56BD76AD66A0101E9
:100EF000456B466B0CC100F10DC101F10EC102F151
:100F00000FC103F110C104F111C105F112C106F1C5
:100F100013C107F114C108F115C109F116C10AF195
:100F200017C10BF135C134F196EF07F002C0E0FFB5
:100F3000005001C0D8FF1000A6B29CEF07F00CC013
:100F4000A9FF0BC0A8FFA69EA69CA684F29E550EE4
:100F5000A76EAA0EA76EA682F28EA694A6B2AEEFD8
:100F600007F00C2A1200A96EA69EA69CA680A85087
:100F70000C2A120004012C0E826FA7EC0AF019EC67
:100F800023F00C50B3EC07F0E8CF00F10C50B3ECB9
:100F900007F0E8CF01F101AFD3EF07F00101FF0E39
:100FA000026FFF0E036FBCEC22F02967DFEF07F042
:100FB0000401200E826FA7EC0AF0E4EF07F00401B1
:100FC0002D0E826FA7EC0AF0E6EC20F01200076A03
:100FD0000F6A106A0F010D0EC16E860EC06E030EF1
:100FE000C26E0F01680E896E130E926E080E8A6E25
:100FF0008A6AF30E936E8B6A900E946EF18EF19E58
:101000000E6A01015B6B5C6B5D6B576B586BF29A00
:101010000101476B486B496B4A6B4B6B4C6B4D6BDB
:101020004E6B4F6B506B516B526B456B466BD76A77
:10103000D66A0F01280ED56EF28A9D90B00ECD6E45
:1010400001015E6B5F6B606B616B626B636B646B0A
:10105000656B666B676B686B696B536B546BCF6AC0
:10106000CE6A0F9A0F9C0F9E9D80760ECA6E9D824F
:1010700002013C0E006FCC6A160EB3EC07F0E8CF0D
:1010800000F1170EB3EC07F0E8CF01F1180EB3EC46
:1010900007F0E8CF02F1190EB3EC07F0E8CF03F147
:1010A000010103AF6EEF08F019EC23F0160E0C6E81
:1010B00000C10BF09CEC07F0170E0C6E01C10BF099
:1010C0009CEC07F0180E0C6E02C10BF09CEC07F0C4
:1010D000190E0C6E03C10BF09CEC07F000C18AF1F5
:1010E00001C18BF102C18CF103C18DF100C18EF100
:1010F00001C18FF102C190F103C191F11A0EB3EC5D
:1011000007F0E8CF00F11B0EB3EC07F0E8CF01F1D8
:101110001C0EB3EC07F0E8CF02F11D0EB3EC07F0A4
:10112000E8CF03F1010103AFC4EF08F019EC23F09D
:101130001A0E0C6E00C10BF09CEC07F01B0E0C6E2F
:1011400001C10BF09CEC07F01C0E0C6E02C10BF001
:101150009CEC07F01D0E0C6E03C10BF09CEC07F02D
:101160001A0EB3EC07F0E8CF00F11B0EB3EC07F05A
:10117000E8CF01F11C0EB3EC07F0E8CF02F11D0E31
:10118000B3EC07F0E8CF03F100C192F101C193F194
:1011900002C194F103C195F1240EAC6E900EAB6EBA
:1011A000240EAC6E080EB86E000EB06E1F0EAF6E41
:1011B0000401806B816B0F01900EAB6E0F019D8A55
:1011C0000301806B816BC26B8B92A9EC29F009EC57
:1011D0002BF089EC27F0200EB3EC07F0E8CF2FF5C9
:1011E00005012F51FF0AD8A4FDEF08F02F6B200E48
:1011F0000C6E2FC50BF09CEC07F00501010E306F53
:101200003C0E316F250EB3EC07F0E8CF00F1260E4F
:10121000B3EC07F0E8CF01F1270EB3EC07F0E8CF0D
:1012200002F1280EB3EC07F0E8CF03F1010103AFA0
:1012300034EF09F019EC23F0250E0C6E00C10BF011
:101240009CEC07F0260E0C6E01C10BF09CEC07F035
:10125000270E0C6E02C10BF09CEC07F0280E0C6EF2
:1012600003C10BF09CEC07F000C153F501C154F52C
:1012700002C155F503C156F500C157F501C158F536
:1012800002C159F503C15AF5290EB3EC07F0E8CFB6
:101290005BF505015C515B5DD8A05BC55CF50501A4
:1012A0002F51020A0EE181B861EF09F005015C2FB0
:1012B0005EEF09F05BC55CF561EF09F081BA48EFBC
:1012C0002BF0210EB3EC07F0E8CF00F1220EB3ECC7
:1012D00007F0E8CF01F1230EB3EC07F0E8CF02F1FD
:1012E000240EB3EC07F0E8CF03F1010103AFA7EF41
:1012F00009F019EC23F0210E0C6E00C10BF09CECF0
:1013000007F0220E0C6E01C10BF09CEC07F0230ECF
:101310000C6E02C10BF09CEC07F0240E0C6E03C1A6
:101320000BF09CEC07F0210EB3EC07F0E8CF00F1D6
:10133000220EB3EC07F0E8CF01F1230EB3EC07F077
:10134000E8CF02F1240EB3EC07F0E8CF03F100C1BF
:101350005DF501C15EF502C15FF503C160F5C0EC4A
:1013600026F082EC25F0D2EC24F005012F51030A7F
:1013700012E005012F51040A1DE005012F51050A55
:1013800024E005012F51060A32E005012F51070A1A
:1013900038E00AEF0AF0ACC500F101010F0E0017AA
:1013A00001010051000A36E001010051050A32E056
:1013B00007EF0AF0ACC500F101010F0E00170101A3
:1013C0000051000A27E007EF0AF00501AC51000ABE
:1013D00021E00501AC51150A1DE00501AC51300AB0
:1013E00019E00501AC51450A15E007EF0AF00501C7
:1013F000AC51000A0FE00501AC51300A0BE007EFD9
:101400000AF00501AC51000A05E007EF0AF081BAC5
:1014100048EF2BF07DEC24F007900001F28EF28C67
:1014200007B067EF1FF00FB048EF1AF00FB80CEFDE
:1014300014F00301805181197F0BD8B467EF1FF0BE
:1014400013EE00F081517F0BE126812BE7CFE8FFFF
:10145000E00BD8B467EF1FF023EE82F0C2513F0BD0
:10146000D926E7CFDFFFC22BDF50780AD8A467EF79
:101470001FF007808EC100F18FC101F190C102F110
:1014800091C103F10101040E046F000E056F000EFF
:10149000066F000E076F1EEC22F000AF59EF0AF046
:1014A0000101030E8E6F000E8F6F000E906F000E05
:1014B000916F03018251720AD8B448EF1AF0825139
:1014C000520AD8B448EF1AF08251750AD8B448EFDE
:1014D0001AF08251630AD8B423EF1CF08251690AD2
:1014E000D8B403EF17F082517A0AD8B416EF18F087
:1014F0008251490AD8B4A2EF16F08251500AD8B4EA
:10150000C0EF15F08251700AD8B403EF16F0825183
:10151000540AD8B42EEF16F08251740AD8B474EF7E
:1015200016F08251730AD8B478EF19F08251530A39
:10153000D8B4DDEF19F082514C0AD8B44DEF0EF05B
:101540008251760AD8B4BBEF0AF058EF1CF00401C0
:1015500014EE00F080517F0BE12682C4E7FF802B60
:10156000120004010D0E826FA7EC0AF00A0E826FC2
:10157000A7EC0AF0120003018351300AD8B4DCEF63
:101580000AF003018351310AD8B413EF0BF00301C1
:101590008351320AD8B4E9EF0BF003018351330AC7
:1015A000D8B4BFEF0CF003018351340AD8B465EF0F
:1015B0000DF0D8A458EF1CF00401760E826FA7EC52
:1015C0000AF00401300E826FA7EC0AF004012C0E21
:1015D000826FA7EC0AF087EC23F019EC23F000C629
:1015E00000F101C601F1BCEC22F030C182F404012B
:1015F000300E8227A7EC0AF031C182F40401300ECC
:101600008227A7EC0AF032C182F40401300E82274F
:10161000A7EC0AF033C182F40401300E8227A7EC54
:101620000AF06DEF14F00401760E826FA7EC0AF059
:101630000401310E826FA7EC0AF004012C0E826FB8
:10164000A7EC0AF0ADEC23F0ADEC23F019EC23F09D
:1016500002C600F103C601F101AF34EF0BF0010146
:10166000FF0E026FFF0E036FBCEC22F029673BEF09
:101670000BF040EF0BF004012D0E826FA7EC0AF087
:101680002FC182F40401300E8227A7EC0AF030C18A
:1016900082F40401300E8227A7EC0AF031C182F4F3
:1016A0000401300E8227A7EC0AF032C182F4040153
:1016B000300E8227A7EC0AF033C182F40401300E09
:1016C0008227A7EC0AF004012C0E826FA7EC0AF027
:1016D00019EC23F004C600F105C601F101AF76EF65
:1016E0000BF00101FF0E026FFF0E036FBCEC22F046
:1016F00029677DEF0BF082EF0BF004012D0E826F56
:10170000A7EC0AF02FC182F40401300E8227A7EC67
:101710000AF030C182F40401300E8227A7EC0AF0EF
:1017200031C182F40401300E8227A7EC0AF032C1E5
:1017300082F40401300E8227A7EC0AF033C182F450
:101740000401300E8227A7EC0AF004012C0E826FF0
:10175000A7EC0AF019EC23F006C600F107C601F168
:1017600001AFB8EF0BF00101FF0E026FFF0E036F28
:10177000BCEC22F02967BFEF0BF0C4EF0BF00401C3
:101780002D0E826FA7EC0AF02FC182F40401300EF7
:101790008227A7EC0AF030C182F40401300E8227C0
:1017A000A7EC0AF031C182F40401300E8227A7ECC5
:1017B0000AF032C182F40401300E8227A7EC0AF04D
:1017C00033C182F40401300E8227A7EC0AF06DEFDA
:1017D00014F00401760E826FA7EC0AF00401320EB9
:1017E000826FA7EC0AF004012C0E826FA7EC0AF0BE
:1017F00015EC24F015EC24F019EC23F008C600F1E8
:1018000009C601F101AF0AEF0CF00101FF0E026FF2
:10181000FF0E036FBCEC22F0296711EF0CF016EFFE
:101820000CF004012D0E826FA7EC0AF02FC182F498
:101830000401300E8227A7EC0AF030C182F40401C3
:10184000300E8227A7EC0AF031C182F40401300E79
:101850008227A7EC0AF032C182F40401300E8227FD
:10186000A7EC0AF033C182F40401300E8227A7EC02
:101870000AF004012C0E826FA7EC0AF019EC23F099
:101880000AC600F10BC601F101AF4CEF0CF00101EB
:10189000FF0E026FFF0E036FBCEC22F0296753EFBF
:1018A0000CF058EF0CF004012D0E826FA7EC0AF03B
:1018B0002FC182F40401300E8227A7EC0AF030C158
:1018C00082F40401300E8227A7EC0AF031C182F4C1
:1018D0000401300E8227A7EC0AF032C182F4040121
:1018E000300E8227A7EC0AF033C182F40401300ED7
:1018F0008227A7EC0AF004012C0E826FA7EC0AF0F5
:1019000019EC23F00CC600F10DC601F101AF8EEF0A
:101910000CF00101FF0E026FFF0E036FBCEC22F012
:10192000296795EF0CF09AEF0CF004012D0E826FF1
:10193000A7EC0AF02FC182F40401300E8227A7EC35
:101940000AF030C182F40401300E8227A7EC0AF0BD
:1019500031C182F40401300E8227A7EC0AF032C1B3
:1019600082F40401300E8227A7EC0AF033C182F41E
:101970000401300E8227A7EC0AF06DEF14F0040189
:10198000760E826FA7EC0AF00401330E826FA7EC8B
:101990000AF004012C0E826FA7EC0AF085C382F4D2
:1019A000A7EC0AF0640E0D6E03018551320A02E1C4
:1019B0006A0E0D6E03018551330A02E1700E0D6E41
:1019C00003018551340A02E1760E0D6E0301855143
:1019D000350A02E17C0E0D6E03018551360A02E1E3
:1019E000820E0D6E03018651780A65E00DC00CF081
:1019F0005AEC23F02981030187512D0AD8B403EF53
:101A00000DF00101299188C32FF189C330F18AC3F8
:101A100031F18BC332F18CC333F167EC23F0DEEC90
:101A200022F000C10BF09CEC07F001C10BF09CEC24
:101A300007F05AEC23F0298103018E512D0AD8B406
:101A400024EF0DF0010129918FC32FF190C330F1E4
:101A500091C331F192C332F193C333F167EC23F0B8
:101A6000DEEC22F000C10BF09CEC07F001C10BF0A2
:101A70009CEC07F05AEC23F02981030195512D0AC3
:101A8000D8B445EF0DF00101299196C32FF197C30A
:101A900030F198C331F199C332F19AC333F167EC55
:101AA00023F0DEEC22F000C10BF09CEC07F001C14A
:101AB0000BF09CEC07F00DC00CF0BAEC07F0BAECA0
:101AC00007F0BAEC07F06DEF14F00401760E826FA8
:101AD000A7EC0AF00401340E826FA7EC0AF00301B0
:101AE0008451780AD8B43DEF0EF03E0E0C6E5AECDD
:101AF00023F02981030185512D0AD8B482EF0DF01E
:101B00000101299186C32FF187C330F188C331F1D8
:101B100089C332F18AC333F167EC23F0DEEC22F0A3
:101B200000C10BF09CEC07F001C10BF09CEC07F03E
:101B30005AEC23F0298103018C512D0AD8B4A3EF6C
:101B40000DF0010129918DC32FF18EC330F18FC3A8
:101B500031F190C332F191C333F167EC23F0DEEC45
:101B600022F000C10BF09CEC07F001C10BF09CECE3
:101B700007F05AEC23F02981030193512D0AD8B4C0
:101B8000C4EF0DF00101299194C32FF195C330F1F9
:101B900096C331F197C332F198C333F167EC23F068
:101BA000DEEC22F000C10BF09CEC07F001C10BF061
:101BB0009CEC07F05AEC23F0298103019A512D0A7D
:101BC000D8B4E5EF0DF0010129919BC32FF19CC31F
:101BD00030F19DC331F19EC332F19FC333F167EC05
:101BE00023F0DEEC22F000C10BF09CEC07F001C109
:101BF0000BF09CEC07F05AEC23F029810301A15172
:101C00002D0AD8B406EF0EF001012991A2C32FF1DD
:101C1000A3C330F1A4C331F1A5C332F1A6C333F19C
:101C200067EC23F0DEEC22F000C10BF09CEC07F037
:101C300001C10BF09CEC07F05AEC23F02981030161
:101C4000A8512D0AD8B427EF0EF001012991A9C39C
:101C50002FF1AAC330F1ABC331F1ACC332F1ADC344
:101C600033F167EC23F0DEEC22F000C10BF09CECCA
:101C700007F001C10BF09CEC07F03E0E0C6EBAECC5
:101C800007F0BAEC07F0BAEC07F0BAEC07F0BAECE0
:101C900007F0BAEC07F06DEF14F003018351300A3E
:101CA000D8B40EEF11F003018351310AD8B41AEF02
:101CB00012F003018351320AD8B486EF12F0030107
:101CC0008351330AD8B494EF12F003018351340ADC
:101CD000D8B4A2EF12F003018351350AD8B411EF42
:101CE00014F003018351360AD8B43FEF14F0030116
:101CF0008351460AD8B465EF13F0030183514D0AAE
:101D0000D8B487EF0FF0030183516D0AD8B4A1EF67
:101D10000FF0030183515A0AD8B494EF11F0030174
:101D20008351490AD8B43FEF15F003018351500A9B
:101D3000D8B471EF14F003018351540AD8B4EAEF18
:101D400014F003018351630AD8B4C1EF0FF003010B
:101D50008351430AD8B4B9EF10F003018351730AD9
:101D6000D8B4BFEF0FF003018351610AD8B4D4EFA8
:101D70000EF003018351650AD8B45CEF11F0030142
:101D80008351450AD8B46AEF11F003018351620A06
:101D9000D8B478EF11F003018351420AD8B486EF2A
:101DA00011F0D8A458EF1CF004014C0E826FA7EC80
:101DB0000AF00401610E826FA7EC0AF082EC25F0B4
:101DC00004012C0E826FA7EC0AF019EC23F0ABC5CE
:101DD00000F10101BCEC22F031C182F40401300EAB
:101DE0008227A7EC0AF032C182F40401300E822768
:101DF000A7EC0AF033C182F40401300E8227A7EC6D
:101E00000AF004012C0E826FA7EC0AF019EC23F003
:101E1000ACC500F10101BCEC22F031C182F4040137
:101E2000300E8227A7EC0AF032C182F40401300E92
:101E30008227A7EC0AF033C182F40401300E822716
:101E4000A7EC0AF004012C0E826FA7EC0AF019EC43
:101E500023F0ADC500F10101BCEC22F031C182F4E8
:101E60000401300E8227A7EC0AF032C182F404018B
:101E7000300E8227A7EC0AF033C182F40401300E41
:101E80008227A7EC0AF004012C0E826FA7EC0AF05F
:101E900019EC23F0AEC500F10101BCEC22F031C118
:101EA00082F40401300E8227A7EC0AF032C182F4DA
:101EB0000401300E8227A7EC0AF033C182F404013A
:101EC000300E8227A7EC0AF004012C0E826FA7ECDB
:101ED0000AF019EC23F0B3C500F10101BCEC22F0CB
:101EE00031C182F40401300E8227A7EC0AF032C11E
:101EF00082F40401300E8227A7EC0AF033C182F489
:101F00000401300E8227A7EC0AF06DEF14F05AECB2
:101F100023F084C333F167EC23F0DEEC22F0200ED3
:101F20000C6E00C10BF09CEC07F000C12FF5050111
:101F30002F51000A06E005012F51010A02E028ECAA
:101F400026F004014C0E826FA7EC0AF004014D0E3E
:101F5000826FA7EC0AF004012C0E826FA7EC0AF046
:101F600019EC23F02FC500F1BCEC22F033C182F450
:101F70000401300E8227A7EC0AF06DEF14F048EF51
:101F80002BF004014C0E826FA7EC0AF00401630EE3
:101F9000826FA7EC0AF0D2EC24F004012C0E826FC1
:101FA000A7EC0AF0D6EC0FF06DEF14F019EC23F06B
:101FB000B1C500F10101003B0F0E0017BCEC22F08F
:101FC00033C182F40401300E8227A7EC0AF0B1C5B8
:101FD00000F101010F0E01010017BCEC22F033C12A
:101FE00082F40401300E8227A7EC0AF004012D0EC2
:101FF000826FA7EC0AF0B0C500F10101003B0F0EA3
:102000000017BCEC22F033C182F40401300E8227A9
:10201000A7EC0AF0B0C500F101010F0E0101001795
:10202000BCEC22F033C182F40401300E8227A7EC0D
:102030000AF004012D0E826FA7EC0AF0AFC500F183
:102040000101003B0F0E0017BCEC22F033C182F4FB
:102050000401300E8227A7EC0AF0AFC500F10101A0
:102060000F0E01010017BCEC22F033C182F4040111
:10207000300E8227A7EC0AF00401200E826FA7EC35
:102080000AF0AEC500F10F0E01010017BCEC22F002
:1020900033C182F40401300E8227A7EC0AF0040158
:1020A000200E826FA7EC0AF0ADC500F1010101011D
:1020B000003B0F0E0017BCEC22F033C182F4040188
:1020C000300E8227A7EC0AF0ADC500F101010F0E1A
:1020D00001010017BCEC22F033C182F40401300E80
:1020E0008227A7EC0AF004013A0E826FA7EC0AF0EF
:1020F000ACC500F10101003B0F0E0017BCEC22F053
:1021000033C182F40401300E8227A7EC0AF0ACC57B
:1021100000F101010F0E01010017BCEC22F033C1E8
:1021200082F40401300E8227A7EC0AF004013A0E73
:10213000826FA7EC0AF0ABC500F10101003B0F0E66
:102140000017BCEC22F033C182F40401300E822768
:10215000A7EC0AF0ABC500F101010F0E0017BCECB3
:1021600022F033C182F40401300E8227A7EC0AF07A
:10217000120084C3E8FF0F0BE83AE8CFB1F585C33E
:10218000E8FF0F0B0501B11387C3E8FF0F0BE83A17
:10219000E8CFB0F588C3E8FF0F0B0501B0138AC381
:1021A000E8FF0F0BE83AE8CFAFF58BC3E8FF0F0B62
:1021B0000501AF138DC3E8FF0F0BE8CFAEF58FC35A
:1021C000E8FF0F0BE83AE8CFADF590C3E8FF0F0B3F
:1021D0000501AD1392C3E8FF0F0BE83AE8CFACF569
:1021E00093C3E8FF0F0B0501AC1395C3E8FF0F0B7A
:1021F000E83AE8CFABF596C3E8FF0F0B0501AB1348
:1022000031EC25F004014C0E826FA7EC0AF00401BA
:10221000430E826FA7EC0AF0CBEF0FF009EC2BF026
:1022200019EC23F02DC500F1BCEC22F004014C0E9A
:10223000826FA7EC0AF00401300E826FA7EC0AF05F
:1022400004012C0E826FA7EC0AF031C182F4040164
:10225000300E8227A7EC0AF032C182F40401300E5E
:102260008227A7EC0AF033C182F40401300E8227E2
:10227000A7EC0AF004012C0E826FA7EC0AF019EC0F
:1022800023F02EC500F1BCEC22F031C182F4040130
:10229000300E8227A7EC0AF032C182F40401300E1E
:1022A0008227A7EC0AF033C182F40401300E8227A2
:1022B000A7EC0AF06DEF14F004014C0E826FA7EC4E
:1022C0000AF00401650E826FA7EC0AF011EC27F00A
:1022D0006DEF14F004014C0E826FA7EC0AF00401BC
:1022E000450E826FA7EC0AF02EEC27F06DEF14F08C
:1022F00004014C0E826FA7EC0AF00401620E826F9B
:10230000A7EC0AF068EC27F06DEF14F004014C0E16
:10231000826FA7EC0AF00401420E826FA7EC0AF06C
:102320004BEC27F06DEF14F004014C0E826FA7EC1C
:102330000AF004015A0E826FA7EC0AF004012C0E79
:10234000826FA7EC0AF009EC2BF019EC23F00501E1
:102350002E51130A06E005012E51170A0DE0C5EFB4
:1023600011F00101000E006F000E016F100E026FE0
:10237000000E036FC5EF11F00101000E006F000E9B
:10238000016F000E026F010E036F0101100E046F4A
:10239000000E056F000E066F000E076F4FEC22F067
:1023A000BCEC22F02AC182F40401300E8227A7EC93
:1023B0000AF02BC182F40401300E8227A7EC0AF048
:1023C0002CC182F40401300E8227A7EC0AF02DC143
:1023D00082F40401300E8227A7EC0AF02EC182F4A9
:1023E0000401300E8227A7EC0AF02FC182F4040109
:1023F000300E8227A7EC0AF030C182F40401300EBF
:102400008227A7EC0AF031C182F40401300E822742
:10241000A7EC0AF032C182F40401300E8227A7EC47
:102420000AF033C182F40401300E8227A7EC0AF0CF
:102430006DEF14F004014C0E826FA7EC0AF004015A
:10244000310E826FA7EC0AF004012C0E826FA7EC0C
:102450000AF025C500F126C501F127C502F128C5FE
:1024600003F10101100E046F000E056F000E066FE0
:10247000000E076F4FEC22F0BCEC22F02AC182F470
:102480000401300E8227A7EC0AF02BC182F404016C
:10249000300E8227A7EC0AF02CC182F40401300E22
:1024A0008227A7EC0AF02DC182F40401300E8227A6
:1024B000A7EC0AF02EC182F40401300E8227A7ECAB
:1024C0000AF02FC182F40401300E8227A7EC0AF033
:1024D00030C182F40401300E8227A7EC0AF031C12A
:1024E00082F40401300E8227A7EC0AF032C182F494
:1024F0000401300E8227A7EC0AF033C182F40401F4
:10250000300E8227A7EC0AF06DEF14F004014C0E98
:10251000826FA7EC0AF00401320E826FA7EC0AF07A
:102520005FEC29F06DEF14F004014C0E826FA7EC04
:102530000AF00401330E826FA7EC0AF0BCEC29F01C
:1025400024EF12F004014C0E826FA7EC0AF0040194
:10255000340E826FA7EC0AF004012C0E826FA7ECF8
:102560000AF05AEC23F084C32AF185C32BF186C309
:102570002CF187C32DF188C32EF189C32FF18AC3B3
:1025800030F18BC331F18CC332F18DC333F10101D2
:10259000296B67EC23F0DEEC22F0100E046F000EC6
:1025A000056F000E066F000E076F2FEC22F000C1C2
:1025B00021F501C122F502C123F503C124F5BCECCC
:1025C0002AF034C5ABF535C5ACF536C5ADF537C524
:1025D000AEF538C5AFF539C5B0F53AC5B1F5D6ECAD
:1025E0000FF004012C0E826FA7EC0AF03BC500F13E
:1025F0003CC501F13DC502F13EC503F10101000EEC
:10260000046F000E056F010E066F000E076F4FEC92
:1026100022F0BCEC22F0296710EF13F015EF13F055
:1026200004012D0E826FA7EC0AF030C182F4040180
:10263000300E8227A7EC0AF031C182F40401300E7B
:102640008227A7EC0AF004012E0E826FA7EC0AF095
:1026500032C182F40401300E8227A7EC0AF033C1A4
:1026600082F40401300E8227A7EC0AF004012C0E3C
:10267000826FA7EC0AF019EC23F03FC500F140C5CA
:1026800001F182EC1DF004012C0E826FA7EC0AF020
:1026900019EC23F041C500F1BCEC22F031C182F409
:1026A0000401300E8227A7EC0AF032C182F4040143
:1026B000300E8227A7EC0AF033C182F40401300EF9
:1026C0008227A7EC0AF06DEF14F05AEC23F085C3D3
:1026D0002AF186C32BF187C32CF188C32DF189C35E
:1026E0002EF18AC32FF18BC330F18CC331F18DC32E
:1026F00032F18EC333F10101296B67EC23F0DEEC7C
:1027000022F00101010E046F000E056F000E066F2E
:10271000000E076F1EEC22F0100E046F000E056F06
:10272000000E066F000E076F2FEC22F000C129F596
:1027300001C12AF502C12BF503C12CF5E8EC28F004
:1027400004014C0E826FA7EC0AF00401460E826F62
:10275000A7EC0AF004012C0E826FA7EC0AF025C545
:1027600000F126C501F127C502F128C503F10101D9
:10277000100E046F000E056F000E066F000E076F3F
:102780004FEC22F0BCEC22F02AC182F40401300E9E
:102790008227A7EC0AF02BC182F40401300E8227B5
:1027A000A7EC0AF02CC182F40401300E8227A7ECBA
:1027B0000AF02DC182F40401300E8227A7EC0AF042
:1027C0002EC182F40401300E8227A7EC0AF02FC13B
:1027D00082F40401300E8227A7EC0AF030C182F4A3
:1027E0000401300E8227A7EC0AF031C182F4040103
:1027F000300E8227A7EC0AF032C182F40401300EB9
:102800008227A7EC0AF033C182F40401300E82273C
:10281000A7EC0AF06DEF14F00F98BCEC29F06DEF07
:1028200014F004014C0E826FA7EC0AF00401350E7F
:10283000826FA7EC0AF004012C0E826FA7EC0AF05D
:1028400019EC23F00784B5C500F10794BCEC22F025
:1028500031C182F40401300E8227A7EC0AF032C1A4
:1028600082F40401300E8227A7EC0AF033C182F40F
:102870000401300E8227A7EC0AF06DEF14F07FEC14
:1028800029F019EC23F033C500F1BCEC22F004016F
:102890004C0E826FA7EC0AF00401360E826FA7EC93
:1028A0000AF004012C0E826FA7EC0AF031C182F409
:1028B0000401300E8227A7EC0AF032C182F4040131
:1028C000300E8227A7EC0AF033C182F40401300EE7
:1028D0008227A7EC0AF06DEF14F0B1EC0AF058EF84
:1028E0001CF004014C0E826FA7EC0AF00401500E9C
:1028F000826FA7EC0AF004012C0E826FA7EC0AF09D
:1029000085C32AF186C32BF187C32CF188C32DF12F
:1029100089C32EF18AC32FF18BC330F18CC331F1FF
:102920008DC332F18EC333F1010167EC23F0DEEC8D
:1029300022F003018451530A0DE0030184514D0A32
:1029400038E00401780E826FA7EC0AF0B1EC0AF0CF
:1029500058EF1CF00401530E826FA7EC0AF0250E0D
:102960000C6E00C10BF09CEC07F0260E0C6E01C142
:102970000BF09CEC07F0270E0C6E02C10BF09CECE8
:1029800007F0280E0C6E03C10BF09CEC07F000C1A1
:1029900053F501C154F502C155F503C156F500C107
:1029A00057F501C158F502C159F503C15AF54EEF6B
:1029B00015F004014D0E826FA7EC0AF0290E0C6E83
:1029C00000C10BF09CEC07F000C15BF500C15CF5A9
:1029D0004EEF15F004014C0E826FA7EC0AF00401D3
:1029E000540E826FA7EC0AF004012C0E826FA7EC44
:1029F0000AF084C32AF185C32BF186C32CF187C367
:102A00002DF188C32EF189C32FF18AC330F18BC316
:102A100031F18DC332F18EC333F1010167EC23F044
:102A2000DEEC22F00101000E046F000E056F010EB6
:102A3000066F000E076F2FEC22F0210E0C6E00C106
:102A40000BF09CEC07F0220E0C6E01C10BF09CEC1D
:102A500007F0230E0C6E02C10BF09CEC07F0240E65
:102A60000C6E03C10BF09CEC07F000C15DF501C1D9
:102A70005EF502C15FF503C160F54EEF15F004018C
:102A80004C0E826FA7EC0AF00401490E826FA7EC8E
:102A90000AF004012C0E826FA7EC0AF0250EB3ECAD
:102AA00007F0E8CF00F1260EB3EC07F0E8CF01F114
:102AB000270EB3EC07F0E8CF02F1280EB3EC07F0D5
:102AC000E8CF03F1BCEC22F09FEC20F00401730E80
:102AD000826FA7EC0AF004012C0E826FA7EC0AF0BB
:102AE00019EC23F0290EB3EC07F0E8CF00F1BCECB1
:102AF00022F09FEC20F00401730E826FA7EC0AF025
:102B000004012C0E826FA7EC0AF057C500F158C5DE
:102B100001F159C502F15AC503F1BCEC22F09FEC5A
:102B200020F00401730E826FA7EC0AF004012C0E52
:102B3000826FA7EC0AF019EC23F05CC500F1BCEC45
:102B400022F09FEC20F004016D0E826FA7EC0AF0DA
:102B500004012C0E826FA7EC0AF05DC500F15EC582
:102B600001F15FC502F160C503F173EC1CF00401D3
:102B70002C0E826FA7EC0AF0B1EC0AF058EF1CF0B3
:102B800083C32AF184C32BF185C32CF186C32DF1B5
:102B900087C32EF188C32FF189C330F18AC331F185
:102BA0008BC332F18CC333F1010167EC23F0DEEC0F
:102BB00022F0160E0C6E00C10BF09CEC07F0170E05
:102BC0000C6E01C10BF09CEC07F0180E0C6E02C1EC
:102BD0000BF09CEC07F0190E0C6E03C10BF09CEC93
:102BE00007F000C18AF101C18BF102C18CF103C170
:102BF0008DF100C18EF101C18FF102C190F103C1CD
:102C000091F1A2EF16F083C32AF184C32BF185C39F
:102C10002CF186C32DF187C32EF188C32FF189C310
:102C200030F18AC331F18BC332F18CC333F101012E
:102C300067EC23F0DEEC22F000C18AF101C18BF1D8
:102C400002C18CF103C18DF100C18EF101C18FF180
:102C500002C190F103C191F1A2EF16F083C32AF1F2
:102C600084C32BF185C32CF186C32DF187C32EF1CC
:102C700088C32FF189C330F18AC331F18CC332F19B
:102C80008DC333F1010167EC23F0DEEC22F001018A
:102C9000000E046F000E056F010E066F000E076F29
:102CA0002FEC22F01A0E0C6E00C10BF09CEC07F01A
:102CB0001B0E0C6E01C10BF09CEC07F01C0E0C6E91
:102CC00002C10BF09CEC07F01D0E0C6E03C10BF063
:102CD0009CEC07F000C192F101C193F102C194F1A3
:102CE00003C195F1A2EF16F083C32AF184C32BF13F
:102CF00085C32CF186C32DF187C32EF188C32FF134
:102D000089C330F18AC331F18CC332F18DC333F101
:102D1000010167EC23F0DEEC22F00101000E046FEC
:102D2000000E056F010E066F000E076F2FEC22F0EC
:102D300000C192F101C193F102C194F103C195F177
:102D4000A2EF16F0160EB3EC07F0E8CF00F1170E65
:102D5000B3EC07F0E8CF01F1180EB3EC07F0E8CFC1
:102D600002F1190EB3EC07F0E8CF03F1BCEC22F04E
:102D70009FEC20F00401730E826FA7EC0AF00401AF
:102D80002C0E826FA7EC0AF08AC100F18BC101F111
:102D90008CC102F18DC103F1BCEC22F09FEC20F05C
:102DA0000401730E826FA7EC0AF004012C0E826FEF
:102DB000A7EC0AF01A0EB3EC07F0E8CF00F11B0EF7
:102DC000B3EC07F0E8CF01F11C0EB3EC07F0E8CF4D
:102DD00002F11D0EB3EC07F0E8CF03F173EC1CF029
:102DE00004012C0E826FA7EC0AF092C100F193C18E
:102DF00001F194C102F195C103F173EC1CF0B1EC47
:102E00000AF058EF1CF00401690E826FA7EC0AF07B
:102E100004012C0E826FA7EC0AF00101040E006F72
:102E2000000E016F000E026F000E036FBCEC22F06B
:102E30002CC182F40401300E8227A7EC0AF02DC1C8
:102E400082F40401300E8227A7EC0AF02EC182F42E
:102E50000401300E8227A7EC0AF02FC182F404018E
:102E6000300E8227A7EC0AF030C182F40401300E44
:102E70008227A7EC0AF031C182F40401300E8227C8
:102E8000A7EC0AF032C182F40401300E8227A7ECCD
:102E90000AF033C182F40401300E8227A7EC0AF055
:102EA00004012C0E826FA7EC0AF001010B0E006FDB
:102EB000000E016F000E026F000E036FBCEC22F0DB
:102EC0002CC182F40401300E8227A7EC0AF02DC138
:102ED00082F40401300E8227A7EC0AF02EC182F49E
:102EE0000401300E8227A7EC0AF02FC182F40401FE
:102EF000300E8227A7EC0AF030C182F40401300EB4
:102F00008227A7EC0AF031C182F40401300E822737
:102F1000A7EC0AF032C182F40401300E8227A7EC3C
:102F20000AF033C182F40401300E8227A7EC0AF0C4
:102F300004012C0E826FA7EC0AF001011C0E006F39
:102F4000000E016F000E026F000E036FBCEC22F04A
:102F50002CC182F40401300E8227A7EC0AF02DC1A7
:102F600082F40401300E8227A7EC0AF02EC182F40D
:102F70000401300E8227A7EC0AF02FC182F404016D
:102F8000300E8227A7EC0AF030C182F40401300E23
:102F90008227A7EC0AF031C182F40401300E8227A7
:102FA000A7EC0AF032C182F40401300E8227A7ECAC
:102FB0000AF033C182F40401300E8227A7EC0AF034
:102FC00004012C0E826FA7EC0AF0200EF86EF76A4F
:102FD000F66A04010900F5CF82F4A7EC0AF00900B3
:102FE000F5CF82F4A7EC0AF00900F5CF82F4A7EC44
:102FF0000AF00900F5CF82F4A7EC0AF00900F5CF3A
:1030000082F4A7EC0AF00900F5CF82F4A7EC0AF0ED
:103010000900F5CF82F4A7EC0AF00900F5CF82F49D
:10302000A7EC0AF0B1EC0AF058EF1CF08351630AE8
:10303000D8A458EF1CF08451610AD8A458EF1CF0B2
:1030400085516C0AD8A458EF1CF08651410A42E021
:103050008651440A1BE08651420AD8B47DEF18F02D
:103060008651350AD8B4E2EF1DF08651360AD8B43D
:1030700037EF1EF08651370AD8B4A0EF1EF0865104
:10308000380AD8B4FEEF1EF058EF1CF00798079AE4
:1030900004017A0E826FA7EC0AF00401780E826FA9
:1030A000A7EC0AF00401640E826FA7EC0AF081A875
:1030B00061EF18F00401550E826FA7EC0AF066EF7D
:1030C00018F004014C0E826FA7EC0AF0B1EC0AF084
:1030D00058EF1CF00788079A04017A0E826FA7EC5C
:1030E0000AF00401410E826FA7EC0AF00401610EA0
:1030F000826FA7EC0AF057EF18F00798078A0401CF
:103100007A0E826FA7EC0AF00401420E826FA7ECE0
:103110000AF00401610E826FA7EC0AF057EF18F075
:10312000010166679BEF18F067679BEF18F068670F
:103130009BEF18F06967B3EF18F04F67A7EF18F02F
:103140005067A7EF18F05167A7EF18F05267B3EF79
:1031500018F00101000E006F000E016F000E026FEB
:10316000000E036F12000101620E046F010E056F65
:10317000000E066F000E076F66C100F167C101F116
:1031800068C102F169C103F11EEC22F003BF37EF01
:1031900019F00101000E046FA80E056F550E066FA1
:1031A000020E076F66C100F167C101F168C102F14B
:1031B00069C103F166C186F167C187F168C188F111
:1031C00069C189F11EEC22F003BFF0EF18F0010194
:1031D000000E866FA80E876F550E886F020E896FDE
:1031E0000E0EB3EC07F0E8CF18F10F0EB3EC07F0BA
:1031F000E8CF19F1100EB3EC07F0E8CF1AF1110E79
:10320000B3EC07F0E8CF1BF167EC21F086C104F1C5
:1032100087C105F188C106F189C107F11EEC22F0D2
:1032200007822BEC21F067EC21F007922BEC21F0C8
:1032300086C100F187C101F188C102F189C103F1A2
:1032400007922BEC21F0CC0E046FE00E056F870E79
:10325000066F050E076F1EEC22F000C118F101C1C8
:1032600019F102C11AF103C11BF16FEF19F001014D
:10327000800E006F1A0E016F060E026F000E036FB4
:103280004FC104F150C105F151C106F152C107F11E
:103290001EEC22F003AF50EF19F019EC23F01200EE
:1032A0000E0EB3EC07F0E8CF18F10F0EB3EC07F0F9
:1032B000E8CF19F1100EB3EC07F0E8CF1AF1110EB8
:1032C000B3EC07F0E8CF1BF14FC100F150C101F1A1
:1032D00051C102F152C103F107822BEC21F018C158
:1032E00000F119C101F11AC102F11BC103F1120071
:1032F0000401730E826FA7EC0AF004012C0E826F9A
:10330000A7EC0AF0078462C166F163C167F164C18A
:1033100068F165C169F14BC14FF14CC150F14DC12C
:1033200051F14EC152F157C159F158C15AF10794A8
:103330009EEC19F0B1EC0AF058EF1CF066C100F1F8
:1033400067C101F168C102F169C103F10101BCEC7F
:1033500022F09FEC20F00401630E826FA7EC0AF0CC
:1033600004012C0E826FA7EC0AF04FC100F150C18E
:1033700001F151C102F152C103F10101BCEC22F093
:103380009FEC20F00401660E826FA7EC0AF00401A6
:103390002C0E826FA7EC0AF019EC23F059C100F152
:1033A0005AC101F10101BCEC22F09FEC20F00401B4
:1033B000740E826FA7EC0AF0120010820401530E03
:1033C000826FA7EC0AF004012C0E826FA7EC0AF0C2
:1033D00083C32AF184C32BF185C32CF186C32DF15D
:1033E00087C32EF188C32FF189C330F18AC331F12D
:1033F0008BC332F18CC333F1010167EC23F0DEECB7
:1034000022F000C166F101C167F102C168F103C198
:1034100069F18EC32AF18FC32BF190C32CF191C3B4
:103420002DF192C32EF193C32FF194C330F195C3C4
:1034300031F196C332F197C333F1010167EC23F008
:10344000DEEC22F000C14FF101C150F102C151F197
:1034500003C152F15AEC23F099C32FF19AC330F112
:103460009BC331F19CC332F19DC333F1010167EC81
:1034700023F0DEEC22F000C159F101C15AF19EECBB
:1034800019F004012C0E826FA7EC0AF04FEF1AF02E
:103490008251520A03E10F824FEF1AF00F928251CC
:1034A000750A03E1108456EF1AF010948251550A00
:1034B00003E110865DEF1AF01096078410B2BAEFA0
:1034C0001AF010A4A6EF1AF0B6C166F1B7C167F101
:1034D000B8C168F1B9C169F1BAC16AF1BBC16BF198
:1034E000BCC16CF1BDC16DF1BEC16EF1BFC16FF168
:1034F000C0C170F1C1C171F1C2C172F1C3C173F138
:10350000C4C174F1C5C175F1C6C176F1C7C177F107
:10351000C8C178F1C9C179F1CAC17AF1CBC17BF1D7
:10352000CCC17CF1CDC17DF1CEC17EF1CFC17FF1A7
:10353000D0C180F1D1C181F1D2C182F1D3C183F177
:10354000D4C184F1D5C185F1AEEF1AF062C166F144
:1035500063C167F164C168F165C169F14BC14FF1A5
:103560004CC150F14DC151F14EC152F157C159F109
:1035700058C15AF107940FA0DCEF1AF001019267CD
:10358000C9EF1AF09367C9EF1AF09467C9EF1AF000
:103590009567CDEF1AF0DCEF1AF090EC18F092C1BD
:1035A00004F193C105F194C106F195C107F11EEC38
:1035B00022F003BF20EF1CF090EC18F00101000E88
:1035C000046F000E056F010E066F000E076F4FECC3
:1035D00022F010A4F3EF1AF00401750E826FA7EC2D
:1035E0000AF0F8EF1AF00401720E826FA7EC0AF0ED
:1035F00004012C0E826FA7EC0AF0BCEC22F02967C4
:1036000007EF1BF00401200E826F0AEF1BF004018C
:103610002D0E826FA7EC0AF030C182F40401300E47
:103620008227A7EC0AF031C182F40401300E822710
:10363000A7EC0AF004012E0E826FA7EC0AF032C14B
:1036400082F40401300E8227A7EC0AF033C182F421
:103650000401300E8227A7EC0AF004016D0E826F80
:10366000A7EC0AF004012C0E826FA7EC0AF04FC100
:1036700000F150C101F151C102F152C103F1010148
:10368000BCEC22F09FEC20F00401480E826FA7EC06
:103690000AF004017A0E826FA7EC0AF004012C0EE6
:1036A000826FA7EC0AF066C100F167C101F168C141
:1036B00002F169C103F10101BCEC22F09FEC20F0A2
:1036C0000401630E826FA7EC0AF004012C0E826FD6
:1036D000A7EC0AF066C100F167C101F168C102F10F
:1036E00069C103F101010A0E046F000E056F000E9F
:1036F000066F000E076F2FEC22F0000E046F120E03
:10370000056F000E066F000E076F4FEC22F0BCEC49
:1037100022F02AC182F40401300E8227A7EC0AF0BD
:103720002BC182F40401300E8227A7EC0AF02CC1D1
:1037300082F40401300E8227A7EC0AF02DC182F436
:103740000401300E8227A7EC0AF02EC182F4040196
:10375000300E8227A7EC0AF02FC182F40401300E4C
:103760008227A7EC0AF030C182F40401300E8227D0
:10377000A7EC0AF004012E0E826FA7EC0AF031C10B
:1037800082F40401300E8227A7EC0AF032C182F4E1
:103790000401300E8227A7EC0AF033C182F4040141
:1037A000300E8227A7EC0AF00401730E826FA7EC9B
:1037B0000AF004012C0E826FA7EC0AF019EC23F03A
:1037C00059C100F15AC101F182EC1DF00FB2ECEFCA
:1037D0001BF00FA01EEF1CF004012C0E826FA7EC53
:1037E0000AF0200EF86EF76AF66A04010900F5CFB8
:1037F00082F4A7EC0AF00900F5CF82F4A7EC0AF0F6
:103800000900F5CF82F4A7EC0AF00900F5CF82F4A5
:10381000A7EC0AF00900F5CF82F4A7EC0AF0090042
:10382000F5CF82F4A7EC0AF00900F5CF82F4A7ECFB
:103830000AF00900F5CF82F4A7EC0AF0B1EC0AF027
:103840000F9058EF1CF00401630E826FA7EC0AF092
:1038500004012C0E826FA7EC0AF05EEC1CF0040150
:103860002C0E826FA7EC0AF0D1EC1CF004012C0E98
:10387000826FA7EC0AF04DEC1DF004012C0E826F54
:10388000A7EC0AF00101F80E006FCD0E016F660E75
:10389000026F030E036F73EC1CF004012C0E826F99
:1038A000A7EC0AF063EC1DF0B1EC0AF058EF1CF045
:1038B0000301C26B0790109267EF1FF0D8900E0EB5
:1038C000B3EC07F0E8CF00F10F0EB3EC07F0E8CF50
:1038D00001F1100EB3EC07F0E8CF02F1110EB3ECDA
:1038E00007F0E8CF03F10101000E046F000E056F31
:1038F000010E066F000E076F4FEC22F0BCEC22F0B9
:103900002AC182F40401300E8227A7EC0AF02BC1F1
:1039100082F40401300E8227A7EC0AF02CC182F455
:103920000401300E8227A7EC0AF02DC182F40401B5
:10393000300E8227A7EC0AF02EC182F40401300E6B
:103940008227A7EC0AF02FC182F40401300E8227EF
:10395000A7EC0AF030C182F40401300E8227A7ECF4
:103960000AF031C182F40401300E8227A7EC0AF07C
:1039700004012E0E826FA7EC0AF032C182F404011A
:10398000300E8227A7EC0AF033C182F40401300E16
:103990008227A7EC0AF004016D0E826FA7EC0AF0F3
:1039A0001200120EB3EC07F0E8CF00F1130EB3ECE7
:1039B00007F0E8CF01F1140EB3EC07F0E8CF02F105
:1039C000150EB3EC07F0E8CF03F101010A0E046F06
:1039D000000E056F000E066F000E076F2FEC22F031
:1039E000000E046F120E056F000E066F000E076FBB
:1039F0004FEC22F0BCEC22F02AC182F40401300E1C
:103A00008227A7EC0AF02BC182F40401300E822732
:103A1000A7EC0AF02CC182F40401300E8227A7EC37
:103A20000AF02DC182F40401300E8227A7EC0AF0BF
:103A30002EC182F40401300E8227A7EC0AF02FC1B8
:103A400082F40401300E8227A7EC0AF030C182F420
:103A50000401300E8227A7EC0AF004012E0E826FBB
:103A6000A7EC0AF031C182F40401300E8227A7ECE2
:103A70000AF032C182F40401300E8227A7EC0AF06A
:103A800033C182F40401300E8227A7EC0AF004014E
:103A9000730E826FA7EC0AF012000A0EB3EC07F067
:103AA000E8CF00F10B0EB3EC07F0E8CF01F10C0EFC
:103AB000B3EC07F0E8CF02F10D0EB3EC07F0E8CF5E
:103AC00003F182EF1DF0060EB3EC07F0E8CF00F132
:103AD000070EB3EC07F0E8CF01F1080EB3EC07F0E6
:103AE000E8CF02F1090EB3EC07F0E8CF03F182EF63
:103AF0001DF0010119EC23F0078457C100F158C1F2
:103B000001F107940101E80E046F800E056F000EAD
:103B1000066F000E076F2FEC22F0000E046F040EEC
:103B2000056F000E066F000E076F4FEC22F0880E37
:103B3000046F130E056F000E066F000E076F1EEC6C
:103B400022F00A0E046F000E056F000E066F000EC5
:103B5000076F4FEC22F0BCEC22F001012967B6EFB1
:103B60001DF00401200E826FB9EF1DF004012D0E2F
:103B7000826FA7EC0AF030C182F40401300E822774
:103B8000A7EC0AF031C182F40401300E8227A7ECC1
:103B90000AF032C182F40401300E8227A7EC0AF049
:103BA00004012E0E826FA7EC0AF033C182F40401E7
:103BB000300E8227A7EC0AF00401430E826FA7ECB7
:103BC0000AF0120087C32AF188C32BF189C32CF1B4
:103BD0008AC32DF18BC32EF18CC32FF18DC330F12D
:103BE0008EC331F190C332F191C333F10101296BDE
:103BF00067EC23F0DEEC22F00101000E046F000EF2
:103C0000056F010E066F000E076F2FEC22F00E0EEF
:103C10000C6E00C10BF09CEC07F00F0E0C6E01C196
:103C20000BF09CEC07F0100E0C6E02C10BF09CEC3C
:103C300007F0110E0C6E03C10BF09CEC07F00401B1
:103C40007A0E826FA7EC0AF004012C0E826FA7ECAB
:103C50000AF00401350E826FA7EC0AF004012C0E65
:103C6000826FA7EC0AF05EEC1CF066EF18F087C3D9
:103C70002AF188C32BF189C32CF18AC32DF18BC3A0
:103C80002EF18CC32FF18DC330F18EC331F190C36F
:103C900032F191C333F10101296B67EC23F0DEECC3
:103CA00022F0880E046F130E056F000E066F000ED3
:103CB000076F23EC22F0000E046F040E056F000E58
:103CC000066F000E076F2FEC22F00101E80E046F63
:103CD000800E056F000E066F000E076F4FEC22F08E
:103CE0000A0E0C6E00C10BF09CEC07F00B0E0C6E74
:103CF00001C10BF09CEC07F00C0E0C6E02C10BF036
:103D00009CEC07F00D0E0C6E03C10BF09CEC07F061
:103D100004017A0E826FA7EC0AF004012C0E826F68
:103D2000A7EC0AF00401360E826FA7EC0AF004013A
:103D30002C0E826FA7EC0AF04DEC1DF066EF18F028
:103D400087C32AF188C32BF189C32CF18AC32DF1D3
:103D50008BC32EF18CC32FF18DC330F18FC331F1A2
:103D600090C332F191C333F1010167EC23F0DEEC33
:103D700022F0000E046F120E056F000E066F000E8B
:103D8000076F2FEC22F001010A0E046F000E056F81
:103D9000000E066F000E076F4FEC22F0120E0C6E35
:103DA00000C10BF09CEC07F0130E0C6E01C10BF080
:103DB0009CEC07F0140E0C6E02C10BF09CEC07F0AB
:103DC000150E0C6E03C10BF09CEC07F004017A0E8B
:103DD000826FA7EC0AF004012C0E826FA7EC0AF0A8
:103DE0000401370E826FA7EC0AF004012C0E826FDB
:103DF000A7EC0AF0D1EC1CF066EF18F087C32AF1AB
:103E000088C32BF189C32CF18AC32DF18BC32EF10A
:103E10008CC32FF18DC330F18EC331F190C332F1D9
:103E200091C333F10101296B67EC23F0DEEC22F042
:103E3000880E046F130E056F000E066F000E076FDD
:103E400023EC22F0000E046F040E056F000E066FC7
:103E5000000E076F2FEC22F00101E80E046F800EB8
:103E6000056F000E066F000E076F4FEC22F0060E76
:103E70000C6E00C10BF09CEC07F0070E0C6E01C13C
:103E80000BF09CEC07F0080E0C6E02C10BF09CECE2
:103E900007F0090E0C6E03C10BF09CEC07F0040157
:103EA0007A0E826FA7EC0AF004012C0E826FA7EC49
:103EB0000AF00401380E826FA7EC0AF004012C0E00
:103EC000826FA7EC0AF063EC1DF066EF18F081A892
:103ED00025EF20F007A8DEEF1FF00101800E006F34
:103EE0001A0E016F060E026F000E036F4BC104F134
:103EF0004CC105F14DC106F14EC107F11EEC22F097
:103F000003BF25EF20F099EC20F04BC100F14CC12C
:103F100001F14DC102F14EC103F107822BEC21F0FA
:103F200018C104F119C105F11AC106F11BC107F14D
:103F3000F80E006FCD0E016F660E026F030E036F59
:103F40001EEC22F00E0E0C6E00C10BF09CEC07F084
:103F50000F0E0C6E01C10BF09CEC07F0100E0C6EF6
:103F600002C10BF09CEC07F0110E0C6E03C10BF0BC
:103F70009CEC07F00784010119EC23F057C100F114
:103F800058C101F107940A0E0C6E00C10BF09CECB5
:103F900007F00B0E0C6E01C10BF09CEC07F00C0E41
:103FA0000C6E02C10BF09CEC07F00D0E0C6E03C101
:103FB0000BF09CEC07F0079825EF20F007AA25EFFF
:103FC00020F00784010119EC23F057C100F158C11A
:103FD00001F10794060E0C6E00C10BF09CEC07F08B
:103FE000070E0C6E01C10BF09CEC07F0080E0C6E76
:103FF00002C10BF09CEC07F0090E0C6E03C10BF034
:104000009CEC07F0078462C100F163C101F164C157
:1040100002F165C103F10794120E0C6E00C10BF0A2
:104020009CEC07F0130E0C6E01C10BF09CEC07F03A
:10403000140E0C6E02C10BF09CEC07F0150E0C6E0A
:1040400003C10BF09CEC07F0079A04018051811921
:104050007F0B0BE09EA809D014EE00F081517F0B7E
:10406000E126E750812B0F01AD6E05012F51010AAA
:1040700013E081AA4CEF20F005012F51000A0AE05D
:104080000FB84CEF20F0050130674CEF20F00FB86F
:104090004CEF20F048EF2BF081B861EF20F082EC7C
:1040A00025F005012F51020A02E061EF20F05C2F9C
:1040B00061EF20F05BC55CF50501010E306F3C0E31
:1040C000316F10EF0AF018C100F119C101F11AC1E6
:1040D00002F11BC103F1000E046F000E056F010E0B
:1040E000066F000E076F4FEC22F029A18EEF20F033
:1040F0002051D8B48EEF20F018C100F119C101F1A0
:104100001AC102F11BC103F1000E046F000E056F0E
:104110000A0E066F000E076F4FEC22F0120001012D
:1041200004510013055101130651021307510313E3
:1041300012000101186B196B1A6B1B6B12002AC15C
:1041400082F40401300E8227A7EC0AF02BC182F41E
:104150000401300E8227A7EC0AF02CC182F404017E
:10416000300E8227A7EC0AF02DC182F40401300E34
:104170008227A7EC0AF02EC182F40401300E8227B8
:10418000A7EC0AF02FC182F40401300E8227A7ECBD
:104190000AF030C182F40401300E8227A7EC0AF045
:1041A00031C182F40401300E8227A7EC0AF032C13B
:1041B00082F40401300E8227A7EC0AF033C182F4A6
:1041C0000401300E8227A7EC0AF012002FC182F4FE
:1041D0000401300E8227A7EC0AF030C182F40401FA
:1041E000300E8227A7EC0AF031C182F40401300EB0
:1041F0008227A7EC0AF032C182F40401300E822734
:10420000A7EC0AF033C182F40401300E8227A7EC38
:104210000AF01200060E116E060E126E060E136ED6
:10422000112E10EF21F0122E10EF21F0132E10EFAF
:1042300021F08B84020E116E020E126E020E136EAE
:10424000112E20EF21F0122E20EF21F0132E20EF5F
:1042500021F08B9412000101005305E1015303E1A9
:10426000025301E1002BEEEC21F019EC23F039515F
:10427000006F3A51016F420E046F4B0E056F000E36
:10428000066F000E076F2FEC22F000C104F101C190
:1042900005F102C106F103C107F118C100F119C10E
:1042A00001F11AC102F11BC103F107B25CEF21F069
:1042B00023EC22F05EEF21F01EEC22F000C118F199
:1042C00001C119F102C11AF103C11BF1120019EC6D
:1042D00023F059C100F15AC101F1060EB3EC07F009
:1042E000E8CF04F1070EB3EC07F0E8CF05F1080EB4
:1042F000B3EC07F0E8CF06F1090EB3EC07F0E8CF16
:1043000007F11EEC22F000C124F101C125F102C128
:1043100026F103C127F1290E046F000E056F000E70
:10432000066F000E076F2FEC22F0EE0E046F430EA7
:10433000056F000E066F000E076F23EC22F024C1FC
:1043400004F125C105F126C106F127C107F12FECC3
:1043500022F000C11CF101C11DF102C11EF103C117
:104360001FF1120EB3EC07F0E8CF04F1130EB3EC1B
:1043700007F0E8CF05F1140EB3EC07F0E8CF06F133
:10438000150EB3EC07F0E8CF07F10D0E006F000E2D
:10439000016F000E026F000E036F2FEC22F0180E5B
:1043A000046F000E056F000E066F000E076F4FECD6
:1043B00022F01CC104F11DC105F11EC106F11FC18F
:1043C00007F123EC22F06A0E046F2A0E056F000E2F
:1043D000066F000E076F1EEC22F01200BF0EFA6E81
:1043E000200E3A6F396BD890003701370237033708
:1043F000D8B0FFEF21F03A2FF4EF21F039073A0758
:104400000353D8B412000331070B80093F6F0339FF
:104410000F0B010F396F80EC5FF0406F390580ECB6
:104420005FF0405D405F396B3F33D8B03927393397
:104430003FA914EF22F040513927120001013EEC50
:1044400023F0D8B01200010103510719346F01ECB9
:1044500023F0D8900751031934AF800F12000101E7
:10446000346B25EC23F0D8A03BEC23F0D8B012003D
:1044700010EC23F019EC23F01F0E366F51EC23F0F3
:104480000B35D8B001EC23F0D8A00335D8B012001A
:10449000362F3EEF22F034B128EC23F01200010158
:1044A000346B04510511061107110008D8A025EC42
:1044B00023F0D8A03BEC23F0D8B01200086B096BB6
:1044C0000A6B0B6B51EC23F01F0E366F51EC23F08F
:1044D00007510B5DD8A479EF22F006510A5DD8A4EC
:1044E00079EF22F00551095DD8A479EF22F004514B
:1044F000085DD8A08CEF22F00451085F0551D8A0C8
:10450000053D095F0651D8A0063D0A5F0751D8A0B6
:10451000073D0B5FD8900081362F66EF22F034B153
:1045200028EC23F0346B25EC23F0D89055EC23F0E5
:1045300007510B5DD8A4A9EF22F006510A5DD8A45B
:10454000A9EF22F00551095DD8A4A9EF22F004518A
:10455000085DD8A0B8EF22F0003FB8EF22F0013F8D
:10456000B8EF22F0023FB8EF22F0032BD8B41200CC
:1045700034B128EC23F012000101346B25EC23F058
:10458000D8B012005AEC23F0200E366F00370137F6
:104590000237033711EE33F00A0E376FE7360A0E93
:1045A000E75CD8B0E76EE552372FCEEF22F0362F1A
:1045B000C6EF22F034B12981D890120001010A0E11
:1045C000346F200E366F11EE29F03451376F0A0E1A
:1045D000D890E652D8B0E726E732372FE9EF22F03D
:1045E0000333023301330033362FE3EF22F0E75079
:1045F000FF0FD8A00335D8B0120029B128EC23F062
:104600001200045100270551D8B0053D012706517D
:10461000D8B0063D02270751D8B0073D0327120046
:104620000051086F0151096F02510A6F03510B6F5E
:1046300012000101006B016B026B036B12000101A0
:10464000046B056B066B076B12000335D8A01200D4
:104650000351800B001F011F021F031F003F38EF93
:1046600023F0013F38EF23F0023F38EF23F0032B14
:10467000342B032512000735D8A012000751800BF8
:10468000041F051F061F071F043F4EEF23F0053FC1
:104690004EEF23F0063F4EEF23F0072B342B072578
:1046A00012000037013702370337083709370A3756
:1046B0000B3712000101296B2A6B2B6B2C6B2D6BB6
:1046C0002E6B2F6B306B316B326B336B1200010131
:1046D0002A510F0B2A6F2B510F0B2B6F2C510F0BE5
:1046E0002C6F2D510F0B2D6F2E510F0B2E6F2F5145
:1046F0000F0B2F6F30510F0B306F31510F0B316F8C
:1047000032510F0B326F33510F0B336F1200899CF4
:10471000000EC76E200EC66E9E96C69EC50EC96E52
:10472000FF0E9EB602D0E82EFCD79E96C69E000EC7
:10473000C96EFF0E9EB602D0E82EFCD7C9CF00F698
:104740009E96C69E000EC96EFF0E9EB602D0E82E43
:10475000FCD7C9CF01F6898C1200000EC76E200E5F
:10476000C66E899C9E96C69EC80EC96EFF0E9EB6EA
:1047700002D0E82EFCD79E96C69E000EC96EFF0E94
:104780009EB602D0E82EFCD7C9CF02F69E96C69EF2
:10479000000EC96EFF0E9EB602D0E82EFCD7C9CF20
:1047A00003F6898C899C9E96C69ECA0EC96EFF0E22
:1047B0009EB602D0E82EFCD79E96C69E000EC96E0D
:1047C000FF0E9EB602D0E82EFCD7C9CF04F69E9607
:1047D000C69E000EC96EFF0E9EB602D0E82EFCD714
:1047E000C9CF05F6898C899C9E96C69ECC0EC96E53
:1047F000FF0E9EB602D0E82EFCD79E96C69E000EF7
:10480000C96EFF0E9EB602D0E82EFCD7C9CF06F6C1
:104810009E96C69E000EC96EFF0E9EB602D0E82E72
:10482000FCD7C9CF07F6898C1200000EC76E200E88
:10483000C66E899C9E96C69EE80EC96EFF0E9EB6F9
:1048400002D0E82EFCD79E96C69E000EC96EFF0EC3
:104850009EB602D0E82EFCD7C9CF08F69E96C69E1B
:10486000000EC96EFF0E9EB602D0E82EFCD7C9CF4F
:1048700009F6898C899C9E96C69EEA0EC96EFF0E2B
:104880009EB602D0E82EFCD79E96C69E000EC96E3C
:10489000FF0E9EB602D0E82EFCD7C9CF0AF69E9630
:1048A000C69E000EC96EFF0E9EB602D0E82EFCD743
:1048B000C9CF0BF6898C899C9E96C69EEC0EC96E5C
:1048C000FF0E9EB602D0E82EFCD79E96C69E000E26
:1048D000C96EFF0E9EB602D0E82EFCD7C9CF0CF6EB
:1048E0009E96C69E000EC96EFF0E9EB602D0E82EA2
:1048F000FCD7C9CF0DF6898C1200000EC76E200EB2
:10490000C66E899C9E96C69E240EC96EFF0E9EB6EC
:1049100002D0E82EFCD79E96C69EE40EC96EFF0E0E
:104920009EB602D0E82EFCD7898C899C9E96C69EA6
:10493000200EC96EFF0E9EB602D0E82EFCD79E96C2
:10494000C69E5F0EC96EFF0E9EB602D0E82EFCD743
:10495000898C899C9E96C69E210EC96EFF0E9EB6BE
:1049600002D0E82EFCD79E96C69EC00EC96EFF0EE2
:104970009EB602D0E82EFCD7898C899C9E96C69E56
:10498000260EC96EFF0E9EB602D0E82EFCD79E966C
:10499000C69E000EC96EFF0E9EB602D0E82EFCD752
:1049A000898C12008984000EC76E220EC66E9E96F8
:1049B000C69E000EC96EFF0E9EB602D0E82EFCD732
:1049C0009E96C69E000EC96EFF0E9EB602D0E82EC1
:1049D000FCD7C9CFABF59E96C69E000EC96EFF0EE2
:1049E0009EB602D0E82EFCD7C9CFACF59E96C69EE7
:1049F000000EC96EFF0E9EB602D0E82EFCD7C9CFBE
:104A0000ADF59E96C69E000EC96EFF0E9EB602D0F4
:104A1000E82EFCD7C9CFAEF59E96C69E000EC96E95
:104A2000FF0E9EB602D0E82EFCD7C9CFAFF59E96FA
:104A3000C69E000EC96EFF0E9EB602D0E82EFCD7B1
:104A4000C9CFB0F59E96C69E000EC96EFF0E9EB6EB
:104A500002D0E82EFCD7C9CFB1F5899485EC27F0B8
:104A600012008984000EC76E220EC66E9E96C69EE8
:104A7000800EC96EFF0E9EB602D0E82EFCD79E9621
:104A8000C69EABC5C9FFFF0E9EB602D0E82EFCD76E
:104A90009E96C69EACC5C9FFFF0E9EB602D0E82EFC
:104AA000FCD79E96C69EADC5C9FFFF0E9EB602D02E
:104AB000E82EFCD79E96C69EAEC5C9FFFF0E9EB6D9
:104AC00002D0E82EFCD79E96C69EAFC5C9FFFF0E4A
:104AD0009EB602D0E82EFCD79E96C69EB0C5C9FFF2
:104AE000FF0E9EB602D0E82EFCD79E96C69EB1C59C
:104AF000C9FFFF0E9EB602D0E82EFCD7899485EC44
:104B000027F012008984000EC76E220EC66E9E9694
:104B1000C69E070EC96EFF0E9EB602D0E82EFCD7C9
:104B20009E96C69E000EC96EFF0E9EB602D0E82E5F
:104B3000FCD7C9CFABF59E96C69E000EC96EFF0E80
:104B40009EB602D0E82EFCD7C9CFACF59E96C69E85
:104B5000000EC96EFF0E9EB602D0E82EFCD7C9CF5C
:104B6000ADF59E96C69E000EC96EFF0E9EB602D093
:104B7000E82EFCD7C9CFAEF5899485EC27F089845F
:104B8000000EC76E220EC66E9E96C69E0F0EC96E92
:104B9000FF0E9EB602D0E82EFCD79E96C69E000E53
:104BA000C96EFF0E9EB602D0E82EFCD7C9CFB3F572
:104BB000899485EC27F012008984000EC76E220EBE
:104BC000C66E9E96C69E870EC96EFF0E9EB602D01A
:104BD000E82EFCD79E96C69EABC5C9FFFF0E9EB6BB
:104BE00002D0E82EFCD79E96C69EACC5C9FFFF0E2C
:104BF0009EB602D0E82EFCD79E96C69EADC5C9FFD4
:104C0000FF0E9EB602D0E82EFCD79E96C69EAEC57D
:104C1000C9FFFF0E9EB602D0E82EFCD7899485EC22
:104C200027F089849E96C69E8F0EC96EFF0E9EB693
:104C300002D0E82EFCD79E96C69EB3C5C9FFFF0ED4
:104C40009EB602D0E82EFCD7899485EC27F012009E
:104C50008984000EC76E220EC66E9E96C69E870E73
:104C6000C96EFF0E9EB602D0E82EFCD79E96C69E59
:104C7000000EC96EFF0E9EB602D0E82EFCD79E969F
:104C8000C69E800EC96EFF0E9EB602D0E82EFCD7DF
:104C90009E96C69E800EC96EFF0E9EB602D0E82E6E
:104CA000FCD79E96C69E800EC96EFF0E9EB602D0A1
:104CB000E82EFCD7899485EC27F089849E96C69EC1
:104CC0008F0EC96EFF0E9EB602D0E82EFCD79E96C0
:104CD000C69E010EC96EFF0E9EB602D0E82EFCD70E
:104CE000899485EC27F012008984000EC76E220E8D
:104CF000C66E9E96C69E870EC96EFF0E9EB602D0E9
:104D0000E82EFCD79E96C69E000EC96EFF0E9EB67C
:104D100002D0E82EFCD79E96C69E000EC96EFF0EEE
:104D20009EB602D0E82EFCD79E96C69E800EC96E17
:104D3000FF0E9EB602D0E82EFCD79E96C69E800E31
:104D4000C96EFF0E9EB602D0E82EFCD7899485EC82
:104D500027F089849E96C69E8F0EC96EFF0E9EB662
:104D600002D0E82EFCD79E96C69E010EC96EFF0E9D
:104D70009EB602D0E82EFCD7899485EC27F012006D
:104D80008984000EC76E220EC66E9E96C69E8F0E3A
:104D9000C96EFF0E9EB602D0E82EFCD785EC27F038
:104DA0009E96C69E810EC96EFF0E9EB602D0E82E5C
:104DB000FCD7899485EC27F08984000EC76E220EFB
:104DC000C66E9E96C69E8F0EC96EFF0E9EB602D010
:104DD000E82EFCD785EC27F09E96C69E010EC96E84
:104DE000FF0E9EB602D0E82EFCD7899485EC27F002
:104DF00089849E96C69E910EC96EFF0E9EB602D005
:104E0000E82EFCD785EC27F09E96C69EA50EC96EAF
:104E1000FF0E9EB602D0E82EFCD7899485EC27F0D1
:104E200012008984000EC76E220EC66E9E96C69E24
:104E30008F0EC96EFF0E9EB602D0E82EFCD785EC11
:104E400027F09E96C69E810EC96EFF0E9EB602D0BA
:104E5000E82EFCD7899485EC27F012008984000E97
:104E6000C76E220EC66E9E96C69E8F0EC96EFF0E30
:104E70009EB602D0E82EFCD785EC27F09E96C69E03
:104E8000010EC96EFF0E9EB602D0E82EFCD78994A3
:104E900085EC27F012008984000EC76E220EC66EC4
:104EA0009E96C69E910EC96EFF0E9EB602D0E82E4B
:104EB000FCD785EC27F09E96C69EA50EC96EFF0E08
:104EC0009EB602D0E82EFCD7899485EC27F012001C
:104ED0008984000EC76E220EC66E9E96C69E910EE7
:104EE000C96EFF0E9EB602D0E82EFCD785EC27F0E7
:104EF0009E96C69E000EC96EFF0E9EB602D0E82E8C
:104F0000FCD7899485EC27F01200050EE82EFED719
:104F100012000501256B266B276B286B899A400EC2
:104F2000C76E200EC66E9E96C69E030EC96EFF0EFD
:104F30009EB602D0E82EFCD79E96C69E27C5C9FF16
:104F4000FF0E9EB602D0E82EFCD79E96C69E26C5C2
:104F5000C9FFFF0E9EB602D0E82EFCD79E96C69ED5
:104F600025C5C9FFFF0E9EB602D0E82EFCD79E963F
:104F7000C69EC952FF0E9EB602D0E82EFCD7898A83
:104F80000F01C950FF0A01E1120005012E51130A59
:104F900005E005012E51170A0CE012000501F00E84
:104FA000256FFF0E266F0F0E276F000E286FE2EFA2
:104FB00027F00501F00E256FFF0E266FFF0E276FFD
:104FC000000E286F899A400EC76E200EC66E9E9600
:104FD000C69E030EC96EFF0E9EB602D0E82EFCD709
:104FE0009E96C69E27C5C9FFFF0E9EB602D0E82E2C
:104FF000FCD79E96C69E26C5C9FFFF0E9EB602D060
:10500000E82EFCD79E96C69E25C5C9FFFF0E9EB60C
:1050100002D0E82EFCD79E96C69EC952FF0E9EB6C1
:1050200002D0E82EFCD7898A0F01C950FF0A1EE082
:1050300005012E51130A05E005012E51170A0CE057
:1050400012000501000E256F000E266F100E276F4F
:10505000000E286FE2EF27F00501000E256F000E0D
:10506000266F000E276F010E286F12000501256BB9
:10507000266B276B286B05012E51130A05E00501ED
:105080002E51170A0CE012000501000E216F000ED0
:10509000226F040E236F000E246F58EF28F00501D5
:1050A000000E216F000E226F800E236F000E246F02
:1050B00021C500F122C501F123C502F124C503F188
:1050C00025C504F126C505F127C506F128C507F158
:1050D0008FEC20F000C125F501C126F502C127F5AE
:1050E00003C128F5899A400EC76E200EC66E9E96A3
:1050F000C69E030EC96EFF0E9EB602D0E82EFCD7E8
:105100009E96C69E27C5C9FFFF0E9EB602D0E82E0A
:10511000FCD79E96C69E26C5C9FFFF0E9EB602D03E
:10512000E82EFCD79E96C69E25C5C9FFFF0E9EB6EB
:1051300002D0E82EFCD79E96C69EC952FF0E9EB6A0
:1051400002D0E82EFCD7898AC950FF0A08E104C1C1
:1051500025F505C126F506C127F507C128F5D89024
:10516000050124332333223321332151F00B216FE6
:105170002167C2EF28F02267C2EF28F02367C2EF51
:1051800028F0246758EF28F00501100E2527E86A5B
:105190002623E86A2723E86A28231200E86A050123
:1051A0002E51130A06E005012E51170A0BE0020EDC
:1051B000120005012851000A03E12751F00B07E016
:1051C000010E120005012851000A01E0010E120033
:1051D00029C500F12AC501F12BC502F12CC503F147
:1051E00025C504F126C505F127C506F128C507F137
:1051F0001EEC22F003BF1200CEEC28F05FE1899A8A
:10520000400EC76E200EC66E9E96C69E060EC96ED6
:10521000FF0E9EB602D0E82EFCD7898A899A9E9608
:10522000C69E020EC96EFF0E9EB602D0E82EFCD7B7
:105230009E96C69E27C5C9FFFF0E9EB602D0E82ED9
:10524000FCD79E96C69E26C5C9FFFF0E9EB602D00D
:10525000E82EFCD79E96C69E25C5C9FFFF0E9EB6BA
:1052600002D0E82EFCD79E96C69E000EC96EFF0E99
:105270009EB602D0E82EFCD7898A899A9E96C69E51
:10528000050EC96EFF0E9EB602D0E82EFCD79E9684
:10529000C69EC952FF0E9EB602D0E82EFCD7C9B0FA
:1052A00047EF29F0898A0501100E2527E86A262391
:1052B000E86A2723E86A2823E8EF28F01200899A91
:1052C000400EC76E200EC66E9E96C69E060EC96E16
:1052D000FF0E9EB602D0E82EFCD7898A899A9E9648
:1052E000C69EC70EC96EFF0E9EB602D0E82EFCD732
:1052F000898A0501256B266B276B286B1200899A1A
:10530000400EC76E200EC66E9E96C69E050EC96ED6
:10531000FF0E9EB602D0E82EFCD79E96C69EC952BE
:10532000FF0E9EB602D0E82EFCD7C9CF33F5898A8E
:105330001200899A400EC76E200EC66E9E96C69EBB
:10534000B90EC96EFF0E9EB602D0E82EFCD7898A30
:105350001200899A400EC76E200EC66E9E96C69E9B
:10536000AB0EC96EFF0E9EB602D0E82EFCD7898A1E
:10537000FF0EE82EFED71200CEEC28F0D8A41200C3
:10538000899A400EC76E200EC66E9E96C69E030E6C
:10539000C96EFF0E9EB602D0E82EFCD79E96C69E22
:1053A00027C5C9FFFF0E9EB602D0E82EFCD79E96F9
:1053B000C69E26C5C9FFFF0E9EB602D0E82EFCD7BA
:1053C0009E96C69E25C5C9FFFF0E9EB602D0E82E4A
:1053D000FCD79E96C69EC952FF0E9EB602D0E82EFE
:1053E000FCD7898A0F01C950FF0AD8A4BBEF2AF065
:1053F0000501FE0E336F0501000E336FD2EC24F071
:10540000ABC534F5ACC535F5ADC536F5AEC537F52C
:10541000AFC538F5B0C539F5B1C53AF50784B6C1A1
:1054200066F1B7C167F1B8C168F1B9C169F14BC1A3
:105430004FF14CC150F14DC151F14EC152F157C124
:1054400059F158C15AF1079490EC18F000C13BF59E
:1054500001C13CF502C13DF503C13EF505015D67A3
:1054600039EF2AF05E6739EF2AF05F6739EF2AF0EB
:1054700060673DEF2AF04BEF2AF05DC504F15EC591
:1054800005F15FC506F160C507F101011EEC22F0D0
:1054900003BFBBEF2AF059C13FF55AC140F5B5C56E
:1054A00041F5B6C542F50501100E326F899A400EDE
:1054B000C76E200EC66E9E96C69E060EC96EFF0E65
:1054C0009EB602D0E82EFCD7898A899A9E96C69EFF
:1054D000020EC96EFF0E9EB602D0E82EFCD79E9635
:1054E000C69E27C5C9FFFF0E9EB602D0E82EFCD788
:1054F0009E96C69E26C5C9FFFF0E9EB602D0E82E18
:10550000FCD79E96C69E25C5C9FFFF0E9EB602D04B
:10551000E82EFCD725EE33F0322F02D09BEF2AF095
:105520009E96C69EDECFC9FFFF0E9EB602D0E82E25
:10553000FCD78CEF2AF0898A899A9E96C69E050E22
:10554000C96EFF0E9EB602D0E82EFCD79E96C69E70
:10555000C952FF0E9EB602D0E82EFCD7C9B0A6EF06
:105560002AF0898A0501100E2527E86A2623E86AB1
:105570002723E86A2823120021C500F122C501F182
:1055800023C502F124C503F1899A400EC76E200E8F
:10559000C66E9E96C69E0B0EC96EFF0E9EB602D0BC
:1055A000E82EFCD79E96C69E02C1C9FFFF0E9EB68E
:1055B00002D0E82EFCD79E96C69E01C1C9FFFF0E01
:1055C0009EB602D0E82EFCD79E96C69E00C1C9FFAB
:1055D000FF0E9EB602D0E82EFCD79E96C69EC952FC
:1055E000FF0E9EB602D0E82EFCD725EE33F0050163
:1055F000100E326F9E96C69EC952FF0E9EB602D006
:10560000E82EFCD7C9CFDEFF322FFAEF2AF0898AC5
:105610001200899A400EC76E200EC66E9E96C69ED8
:10562000900EC96EFF0E9EB602D0E82EFCD79E9655
:10563000C69E000EC96EFF0E9EB602D0E82EFCD7A5
:105640009E96C69E000EC96EFF0E9EB602D0E82E34
:10565000FCD79E96C69E000EC96EFF0E9EB602D067
:10566000E82EFCD79E96C69EC952FF0E9EB602D06B
:10567000E82EFCD7C9CF2DF59E96C69EC952FF0EC7
:105680009EB602D0E82EFCD7C9CF2EF5898A12002B
:105690000AEC21F0B5C5E8FFD70802E30AEC21F0D7
:1056A000B5C5E8FFC80802E30AEC21F0B5C5E8FF7C
:1056B000B90802E30AEC21F0B5C5E8FFAA0802E345
:1056C0000AEC21F0B5C5E8FF9B0802E30AEC21F0E3
:1056D00082EC25F099EC29F0F29CF29E8B94899C47
:1056E000C69AC290898C9482948C720ED36ED3A485
:1056F000FED789968A909390FF0EE8CF00F0E82EAF
:10570000FED7002EFCD78150F294F29A9E909D9085
:105710009E929D92F298F292F290F286F28E03009F
:02572000FF0088
:10BF0000E844F926000C160C2B0C3F0C520C640C68
:10BF1000760C860C960CA50CB30CC10CCF0CDC0C6B
:06BF2000E80CF40C000C1B
:00000001FF
